:1000000028288F018E00FF308E07031C8F07031CEA
:10001000232803308D00DF300F2003288D01E83EB8
:100020008C008D09FC30031C18288C070318152838
:100030008C0764008D0F15280C181E288C1C222894
:1000400000002228080083130313831264000800B1
:1000500010308500831685018312C0308600831618
:100060003F30860083120608A6000730A60564000C
:100070002608003C031D3F28C03086003328053089
:1000800001200608A6000730A60564002608003CEB
:100090000319332864002608043C03195E28640011
:1000A0002608013C0319622864002608023C031953
:1000B000682864002608033C03196128851405128A
:1000C0008428861306136400061E332805147B2833
:1000D00086136400061E33286400861E73283A3097
:1000E0008F00983002203A308F0098300220640050
:1000F000061E332805146400861D81288515051504
:0C0100007B28851105117B2885158428BB
:02400E00F53F7C
:00000001FF
